:020000020000FC
:1000000058CDA4C1000000001FC000008DC000003A
:10001000000097C00000000000000000020304067A
:10002000080C10182030406080000406080C1018DE
:100030002030406080A0C0000003070F1F000505AE
:100040000D050305030302004FB662FD0CC05520E9
:1000500041F00994C52DC095089483FDC795C4BD92
:1000600064604FBE1895C0916400089483FDC795E5
:10007000C4BD6B7FC0916400CF3F09F41EC070FF08
:100080001AC082FD05C04FBE91989098939818951C
:1000900076FD0EC065FD0CC0C091B100C0FD949806
:1000A000C1FD9798C2FD9598CAEFC095CA95F1F722
:1000B0009198909893984FBE189524BCCC27C06413
:1000C000C8BF6460F8CFC6CF70FFC4CF65FDC2CF94
:1000D000919AC0CF70FFBECF65FDBCCF909ABACFCA
:1000E00070FFB8CF65FDB6CF939AB4CF949A70FFE6
:1000F000B1CF65FDAFCFC7E0CA95F1F7919AAACF0E
:10010000979A70FFA7CF65FDA5CFC7E0CA95F1F715
:10011000909AA0CF959A70FF9DCF65FD9BCFC7E0C9
:10012000CA95F1F7939A96CF4FB6C9B7CF7EC9BF9C
:100130006E7FCCB5CE0DDDB5DF1DDBBDCABD4FBEBC
:1001400018953FB68F7EABB7A074A2118061A0E076
:10015000ABBFA9B7AE7FA9BF7894A0916800AA23CE
:1001600041F085FD2AC0A0916800AA95A09368007F
:1001700024C040E050E085FD14C0A0B396FFA095D8
:10018000A2FD4FEFA3E096FFA2E0A5BFAA27A064BF
:10019000AABF8D7FA0B396FFA095A2FD5FEF451784
:1001A00041F7A8E161FDA093680085FD03C0A8E1C7
:1001B000A093680040939600816085FD0EC0A091D9
:1001C0006900AA2331F0A0916900AA95A093690063
:1001D00004C08061AA27A064AABF80FF3DC0A0918F
:1001E00096004A2F61FF8E7F85FD18C0403F08F0C2
:1001F00040EFA42FA295AF704A0F5091B600533034
:1002000069F0A695A69550FD01C0A69552FD03C0C4
:10021000A41B4A2F03C04A0F08F44FEFA0919F0080
:100220004A1708F44A2F40936100A72FA670A1F047
:1002300073FD12C0A0917000AA0FAA0F50919E00EA
:1002400056955695541708F0452F4A0F4093610074
:1002500018F4AFEFA0936100A0916100A093630038
:1002600040916300A0919B004A1708F04A2F542E3A
:10027000A091A000AA2309F422C0542F5A1B10F405
:10028000A42F50E0BA2E8894AA1FAA2EA091A200F3
:10029000A095AA22A50E58F0A091A100A21509F0E0
:1002A000AA95AA0EA093A10048F04A2D08C0A091DB
:1002B000A100BA1608F0A395A093A1004FEF4093B8
:1002C00064007F7B485F08F07064A52DA03408F0BF
:1002D0006860A0916000A395A093600051F0F8942D
:1002E000A9B7A160A9BF84FF02C0A0E4ABBF3FBE15
:1002F0001895A0917400A395A093740041E05091CB
:100300006800552329F085FF03C05A955093680073
:10031000A0919600A13018F0209299000DC0209273
:100320009A002092A300A0919900AF5FA09399003A
:1003300018F0AFEFA0939900F894A9B7A160A9BFF6
:1003400084FF02C0A0E4ABBF3FBE18953FB64CB5DA
:100350005DB58F7EABB7A074A2118061A0E0ABBF8A
:10036000A9B7AE7FA9BF789481FD23C0A2E096FF14
:10037000A3E0A5BF8260A0B396FFA095A2FF05C031
:1003800040936500509366003EC1A3E096FFA2E053
:10039000A5BFAA27A064AABF8D7F85FF01C026C183
:1003A00040E0A0B396FFA095A2FD20C14093960027
:1003B0000FC1A3E096FFA2E0A5BF8D7F61FF71C0D2
:1003C000A2E096FFA3E0A5BFAA27A064AABF82600F
:1003D0004093910050939200A0908F004A19B090E2
:1003E00090005B09BB24A22C4C38520518F42092D3
:1003F000950049C0A091D400AA2359F1483C520568
:1004000028F4A0E1BA2EAAE0AA2E23C04836A1E023
:100410005A0728F4A8E0BA2EAFE0AA2E1AC0403D31
:10042000A2E05A0728F4A4E0BA2EAEE1AA2E11C029
:10043000403AA5E05A0728F4A2E0BA2EACE3AA2E6F
:1004400008C04839A8E05A0720F4A1E0BA2EA8E76E
:10045000AA2EC42EA0919300CA1AD52EA091940062
:10046000DA0ADD202AF4AFEFC094D094CA1ADA0A6F
:1004700020929500A8E0A210A0E0CA14DA0618F4B1
:10048000A1E0A09395004093930050939400409175
:1004900091005091920040938F005093900042E061
:1004A00097C0A09165004A1BA09166005A0B94FD6D
:1004B00082C093FD80C092FD7CC086FF03C0D52E14
:1004C000C42E0CC05695479591FD73C0569547951F
:1004D00090FD6FC0D52EC42ED694C79461FD19C06F
:1004E000AC2DAC51AD2DA24008F005C0DD2089F443
:1004F000AC2DA85C70F4A0916700A395AA2311F01D
:10050000A0936700AA3008F471C020929600816021
:100510006DC0A0916700AA2319F0AA95A093670067
:10052000A22C5091BA0097FD06C0A090C80053308D
:1005300011F4A090D000AAEFAA0EA22DA21DCA18F5
:10054000DA0A4FB74170533049F4442321F087FD54
:1005500005C0806803C087FF01C08F77442359F02E
:10056000533031F4AFEFC094D094CA1ADA0A03C002
:1005700040E050E020C0533049F4CC0CDD1CAAE030
:10058000CA1AD20818F4A0E0CA2ED22CAFEFCA16AD
:10059000D20418F04FEF50E00EC0A091AC00CA9EFC
:1005A000412D000C441F50E008F012C04FEF50E006
:1005B0000FC05695479594FF07C0552309F04FEF9C
:1005C000A42FA6954A0F521D4F3F520508F04FEF3A
:1005D00040939600816061FF09C0AFE1A095A92317
:1005E000AB299A2F8F7DBB2009F48062A8E1A093EC
:1005F000680085FF03C0AAE0A093680061FD03C006
:1006000085FD01C08F7E85FD03C0A6E0A093690033
:10061000F894A9B7A160A9BF84FF02C0A0E4ABBF52
:100620003FBE189511E00AC013E008C01AE006C0EA
:100630001EE104C014E602C018EC00C005E1BB27AF
:10064000BA95F1F70A95D9F71A95C1F708952AE3F3
:1006500038E709C020E33CE806C02AE234EB03C0D7
:1006600025E238EC00C012E0BB27979ABA95F1F763
:10067000909ABA95F1F79098BA95F1F79798BA953C
:10068000F1F7123009F0919A123009F4939AB0916F
:10069000AD00BA95F1F7123009F09198123009F4D3
:1006A0009398B7E8BA95F1F71A95F1F6022FB22FA1
:1006B000BA95F1F70A95D9F73A95A9F6979A089558
:1006C000221B39E0001F3A9509F40895221F211BCF
:1006D00018F4210F8894F6CF0894F4CF622C722C72
:1006E000B0E08894B395221F331FE0F73795279524
:1006F0008894912E802E020B130B10F4192D082DC7
:1007000010F4889401C00894661C771CBA9571F7A0
:10071000172D062D0895322D11232AF43A950095B0
:100720001095031B130BF894029F712C002D129F40
:10073000912C802C7894780C172D921C292DB4E0E4
:100740006B2E2695179507956A94D9F7332321F0D8
:1007500000951095031B130B0895089510917B00CD
:10076000169500917A000795B0917E00B01B0B2F73
:10077000B0917F00B10B1B2F28F40038BFEF1B078F
:1007800040F009C00F37120508F405C00FE710E06C
:1007900002C000E81FEF00938300109384000895C7
:1007A00000918300B09180000B0F10918400B091F4
:1007B00081001B1F20E03091840033230AF42A9526
:1007C000B09182002B1F1AF4203F40F00AC02F3056
:1007D00008F407C00FEF1FEF2FE003C000E010E0A8
:1007E00020EF30916300B0919B003B1718F432303A
:1007F00030F009C0B0918400BB235AF004C0B0911E
:100800008400BB2332F40093800010938100209376
:10081000820008952091D70000918300000F10916D
:100820008400111F78DF11232AF40038BFEF1B0763
:1008300040F009C00F37120508F405C00FE710E0BB
:1008400002C000E81FEF002352F0B0916200B01B1D
:100850000B2F18F0013008F00AC001E008C0009525
:100860000F5FB09162000B0F08F001C00FEF009313
:10087000850008952091D800009181001091820098
:100880004ADF11232AF40130BFEF1B0740F009C0F3
:100890000F3F120508F405C00FEF10E002C001E0A1
:1008A0001FEF112352F0B0918500B01B0B2F18F0F1
:1008B000013008F00AC001E008C000950F5FB09158
:1008C00085000B0F08F001C00FEF0093630008953F
:1008D0000FEF677F71FD29C072FD09C06860B0919C
:1008E0007B00BA3020F0B52DB03408F4677FB091AA
:1008F000D300BB23D1F0B0917B00BB23B1F00FEF4D
:1009000010917B00DDDEF894B091730072FDB5E0CC
:100910000B9F112D002D7894112309F00FEFB0914A
:100920009E000B1710F400919E0000939D00089507
:1009300000917A0010917B0000541140B0919D000D
:1009400010F4BA9501C0B39511F0B0939D000895CD
:1009500000C008952091B500B6B1B6FDFBCF04B13B
:1009600015B1B6B1BF77B6B9B091AA00B395B0933F
:10097000AA00B83060F12092AA00B091D200BB2347
:1009800021F1112329F0B091AB00BF3F61F009C004
:10099000B091AB000B1739F020F4BB2321F0BA95CE
:1009A00002C0B395E1F300919B00B093AB00B0306F
:1009B00050F400ECB03038F400E8B03020F400E43B
:1009C000B03008F400E000939B007F7E0895B09162
:1009D0009B00B39511F0B0939B00B091AA00B73083
:1009E00009F47061089502E3F894B091D9000B9F67
:1009F000012D000C001F7894B0919B000B1710F094
:100A000000919B000093610000936300502E0093BF
:100A1000640000939E00089520927A00B0EFB09396
:100A20007B000895F8940CB51DB52091740078945E
:100A300030917500609076000093750010937600F9
:100A4000031B160971FD03C077FD7DC027C07090A0
:100A50007700209377002709222311F00FEF1FEF73
:100A600080907800909079003093780060927900BF
:100A700000917500109176000819190920917A00EB
:100A800030917B0036952795020F131F10F40FEF5E
:100A90001FEF00937A0010937B0029C020917A0009
:100AA00030917B003901B4E08B2EB2E09B2E3430C4
:100AB00010F08A949A94383010F08A949A9476942C
:100AC00067948A94E1F726193709992021F0169541
:100AD00007959A94E1F7200F311F20937A00309305
:100AE0007B0028F43FEF30937A0030937B00323064
:100AF00008F4706871FF02C0B3E00DC0B091C4008B
:100B000000917100023838F0B395003A08F0B395BF
:100B1000B63008F0B5E09B2EB4E08B2E10917B0030
:100B200000917A0024E0169507952A95E1F70819B7
:100B3000120928F0B02FB250B12FB20910F402E020
:100B400010E0980126C020917A0030917B00390195
:100B5000769467946694669466942619320906958D
:100B60000695200F321D20937A0030937B0032309F
:100B700008F07F7704E036952795369527952695DA
:100B80002695201B10F0223008F422E08901909075
:100B9000C40060FDFECFE0908B00F0908C0061609F
:100BA000B9B7B061B9BF380177FD41C07694679499
:100BB00000938B0010938C00B92DB330E1F0B0FDA1
:100BC00004C0060D171D930106C0000F111F02502F
:100BD000120922E030E0B92DB33068F020938D0087
:100BE00030938E00009387001093880060928900F4
:100BF00070928A003AC000938D0010938E0020936B
:100C00008700309388006092890070928A0071FF9B
:100C10000DC0BFE0B0938D0020928E00B09389008C
:100C200020928A00B0938B0020928C001EC06694A4
:100C300000938B00B92DB33091F0B0FD03C0060DC9
:100C4000262D03C0000F025022E0B92DB33038F03A
:100C500020938D00009387006092890006C0009366
:100C60008D00209387006092890000917C0002FD36
:100C70000350013031F495FD0CC0B2E0B06CB7B94F
:100C80000BC0023021F4B3E0B06CB7B905C095FDDC
:100C9000F4CFB4E0B06CB7B90091A200000F10F42B
:100CA000BBE60B270093A20060FDFECFB2E0B0933D
:100CB0006E006160B9B7B061B9BFB72FB670D1F03F
:100CC00020917A0030917B003695279536952795AF
:100CD00071FF02C0B0E43B0FF8940CB51DB5020FD4
:100CE000131F1BBD0ABD6160B0E1B8BFB9B7B061E9
:100CF000B9BF78940895606120927D0020E067FD7F
:100D000020E206C0606120927D0020E267FD20E0C5
:100D100001E011E077FD11C0B72FB67009F06F7ECA
:100D200014E100917B00069509F403950F3008F05B
:100D30000FE071FF02C004E114E160FD0FC0B0914B
:100D40007D00BB2359F071FF06C0B0916E00BA95CB
:100D5000B0936E0011F4706247C0ABDFB0B7B77FDD
:100D6000B0BFB8B1B0B7B860B0BFB0917D00B395B7
:100D7000B0937D00B8B177FD06C0B1E071FDB3E07E
:100D8000BA95F1F7B8B1B072B21709F022C071FF8D
:100D900005C00395011708F00A95CFCF64FD05C083
:100DA0000395011708F0B4CFC8CF6F7EF8943CB517
:100DB0006DB470907A0080907B00370D681C6BBC1E
:100DC0003ABD6160B0E1B8BFB9B7B061B9BF78945E
:100DD0009FCFB0916D00B13008F49ACF64FD98CFE9
:100DE0000A9509F0AACF7F7D20918D0030918E0069
:100DF000F894B0E1B8BF0CB51DB5020F131F1BBDB1
:100E00000ABDE0908700F09088006160B9B7B061DA
:100E1000B9BF7894B72FB67039F0B0916D0072FFFA
:100E2000B395B0936D0009C075FF07C067FD05C09D
:100E300064FD03C0BF91BF91F0C4089500E063FF5B
:100E400003C064FF01C001E0F89410917100B7E0A5
:100E50001B9F212D102D7894200F269517952695F0
:100E600017952695179510937100183718F4B8E761
:100E7000B093710000917100B09172000B1720F0D7
:100E8000606291989098939860FDFECFE090890001
:100E9000F0908A006160B9B7B061B9BF0895B2E05F
:100EA00095FD0AC0F894B0937C00979A949862FFDD
:100EB00001C0939A7894F4C0F894B0937C00979A08
:100EC000959862FF01C0919A7894EAC0B3E082FFDE
:100ED00024C095FD11C002E0F894B0937C00E0E8D6
:100EE000F0E00093B1009398959A62FF02C0909A47
:100EF00001C097987894D4C002E0F894B0937C0035
:100F0000E0E8F0E00093B1009198949A62FF02C08B
:100F1000909A01C097987894C3C095FD0BC0F8943F
:100F2000B0937C00EAE6F0E0939862FF01C0909AEB
:100F30007894B6C0F894B0937C00EAE6F0E091981B
:100F400062FF01C0909A7894ABC0B4E095FD0AC0EE
:100F5000F894B0937C00949A959862FF01C0909A9F
:100F600078949EC0F894B0937C00959A949862FF10
:100F700001C0909A789494C0B5E082FF24C095FD9A
:100F800011C001E0F894B0937C00E6E7F0E0009334
:100F9000B1009098979A62FF02C0919A01C094980C
:100FA00078947EC004E0F894B0937C00EAE8F0E026
:100FB0000093B1009098979A62FF02C0939A01C083
:100FC000959878946DC095FD0BC0F894B0937C0013
:100FD000E4E6F0E0909862FF01C0919A789460C0D6
:100FE000F894B0937C00E0E7F0E0909862FF01C0D5
:100FF000939A789455C0B6E095FD0AC0F894B093E2
:101000007C00959A979862FF01C0919A789448C0A5
:10101000F894B0937C00949A979862FF01C0939AD9
:1010200078943EC0B1E082FF24C095FD11C004E079
:10103000F894B0937C00EAE8F0E00093B100919856
:10104000949A62FF02C0939A01C09598789428C040
:1010500001E0F894B0937C00E6E7F0E00093B10083
:101060009398959A62FF02C0919A01C094987894DF
:1010700017C095FD0BC0F894B0937C00E0E7F0E05A
:10108000919862FF01C0939A78940AC0F894B09343
:101090007C00E4E6F0E0939862FF01C0919A7894B6
:1010A0006F7D089523E630E0F9012092B100919818
:1010B00090989398949A979A959A6B7F0895A2EB3B
:1010C000B0E00FEF0D930D930D930D9303E00D938F
:1010D00004E00D930AE00D9303E00D9301E00D93FE
:1010E00001E00D93AEEBB0E001E00D930FEF0D9337
:1010F0000D930D930D930D9303E00D930FEF0D934F
:101100000FEF0D930D9305E20D9300ED0D930AEF94
:101110000D930AEF0D9304E00D930FEF0D9301E093
:101120000D9300E00D930AE70D930FEF0D9300E090
:101130000D9301E00D9300E00D9303E00D9300E0AB
:101140000D9308952091B9008B7F233009F48460BA
:10115000B091BA00B33019F09F7DB1FD90629F7BD2
:10116000B091BB00B1FD9064223011F0886001C0E5
:10117000877F08950A95E00FF21DB4910895ECE180
:10118000F0E00091B200F6DFB093D700ECE1F0E0C0
:101190000091B300EFDFB093D800EAE2F0E00091F5
:1011A000B800E8DFB093D9000091B800023008F42D
:1011B00002E000937300B091CE000FEFB23009F45B
:1011C00000EAB33009F402E800937200E8E3F0E0CB
:1011D0000091D500CFDFB093A0000895089520912D
:1011E000C8003091C900B091BA00B33009F43E5044
:1011F00097FF02C020E03FEFB32FB21B6B2EB25817
:1012000010F4B2E86B2E00E00395609EB12DBD573F
:10121000D8F30093AC0008959068E1DF09DA20E08C
:1012200030E0B0E16B2E00DAB09196002B0F321D4A
:101230006A94C9F7B4E036952795BA95E1F7822EFE
:101240009F77CDDF0895F894E3E0F0E0B9E0B7BF11
:10125000B491B078C1F3F894A895B1B5B861B1BDB7
:10126000B0E0B1BDB4E0BEBFBFE5BDBF1BDFB0E0C5
:10127000B8BBB0E1B7BBB0E0B5BBB0E0B4BBB0EB5E
:10128000B2BBBBEBB1BB2224A0E0B0E02D92AA31EF
:10129000E9F7A0E6B0E00FEF2D920A95E9F7B1E08B
:1012A000B093A2000CDFF5D2B7E0B06CB7B9B6B11D
:1012B000B460B068B6B90091CA000093AD00B1E067
:1012C000B0936A00F894B8D9C2D9B2D9C3D9B0D909
:1012D000C4D9AED965D3B0D9AFD9ACD9F8940AEF97
:1012E0001AEFA0B396FFA095A2FF1FC01A95C9F7E9
:1012F0000A95B1F7E0E0FCE1B591B43E39F4B5915F
:10130000B03E21F4B591BF3F09F40CC0E0E0F39585
:10131000F395B591B83F49F4B591B43931F4B5912D
:10132000BA3A19F4EE27F69509940CDF28DF56DF58
:1013300056DF0091CA000093AD00B4DEB2E0B3BF47
:10134000B2E0BEBDB2E0B5BDB1E5B8BFB9BFB0B7A0
:10135000B77FB0BFB8B1B0B7B860B0BF63D9789449
:10136000F7DA20927000B3E096FFB2E0B5BFB0E4C8
:10137000BBBFBB27B064BABF8D7F5ED9626033E06C
:101380002CE0B0919500BB2321F42CE03A9509F4B0
:10139000A5CF4ED980FFA2CF8E7FB0919600B230FC
:1013A00078F3B92FBF710091980000939700B09324
:1013B0009800B01729F72A9521F76D7FB3E096FFC3
:1013C000B2E0B5BFBB27B064BABF8D7FB091D40087
:1013D000BB2321F48062B92FB0709B2F8F7B2092AA
:1013E000670028D985FF05C0B0916700BA3008F0C2
:1013F00080641AD902E085FF01C000E0B091960038
:10140000B017B8F3F89423D922D921D9789414D9F4
:1014100020928600B091BA00B33009F474C004D9A8
:10142000B091BE00B13008F46EC0B0916A00B13026
:1014300008F469C085FD18C0B0919600BF3F08F45C
:1014400062C0F8940DD97894F5D8B0919600B13077
:10145000C0F7F894FCD8EAD8FAD87894EBD8B091D1
:101460009600BF3FB0F3CEC2B8E09B2E9068F894D0
:10147000B6DE7894DFD8F8949F77B1DE809096003E
:10148000B0919600BF37789408F445C0CBD8F89453
:10149000E7D878949A9451F7BFDEB82DB550B09341
:1014A000C900CAD8F89422D280D27894BAE09B2E90
:1014B0009068F89494DE7894BDD8F8949F778FDE86
:1014C00080909600B0919600BF37789478F7AAD8AC
:1014D000F894BDD8ABD8BBD878949A9449F79CDEE1
:1014E000B82DBB5FB093C800A7D8F894FFD16CD2D9
:1014F0007894A0D8F89473DE7894B0919600BF3FAA
:1015000008F498CF7FC200919600B09186000B1727
:1015100010F0009386008ED801E0B091BA00B3506D
:1015200009F405E0B0919600B01708F073CFF89475
:1015300097D896D895D878947FD820926A00209230
:101540006B0020926C00B0916B00B395B0936B0070
:10155000BF3F71F5B0916C00B395B0936C00B09142
:10156000CC0009E1BA9559F002E3BA9541F00DE7D4
:10157000BA9529F00AEFBA9511F020926C00B0915B
:101580006C00B017A8F08EDD4DD8B0916C00BA9504
:10159000B0936C0020926B00B091CB00B093AD0083
:1015A000F8945ED87894B091CA00B093AD0042D858
:1015B0003DD8B0916800BB2319F485FF01C08ECEE1
:1015C00001E085FD01C006E0B0919600B01708F477
:1015D000BACFB091BA00B35009F02CD8B0916800DE
:1015E000BB2309F47BCEF8945DDD2092610020924C
:1015F000620020926300522C209264002092A1008D
:101600007894B091B700BB0FB0939F0020927E00FA
:1016100020927F0020928000209281002092820000
:101620002092AA0060E070E020927100B8E0B093D0
:10163000AA007061F7D7B7E074FDB7E0B06CB7B936
:10164000B6B1B068B064B6B9B6B1B6FDFDCF04B1FD
:1016500015B1B6B1BF77B6B9112309F00FEF0093FA
:10166000AB0078D9B8E0B093AA0070616BDDF89454
:10167000BFEFB0939B00B7D9B0916100B0939B00CE
:10168000B0939C00B0939D007894B1E0B09361005A
:10169000B09363005B2EB0936400B093A400B0914C
:1016A0009A00B093A300B091BA00B33019F49F7DB3
:1016B00087FD90627160726020926D009CDCB2DCEC
:1016C000ABD9B0D9A9D9AED9A7D91CDB46D8B6DBDE
:1016D000E6DBA8D910DB66FD41D877FFF9D877FDA6
:1016E00027D9ACDBF3DB9ED90DDB66FD59D8A6DB31
:1016F0002CDC98D900DB66FD8DD8A0DB3DDC92D9CF
:1017000001DB66FDB7D89ADB76DC8CD9F4DAB7E07A
:1017100074FDB7E0B06CB7B9B6B1B068B064B6B933
:101720008DDB80DC7FD916D971FF21C0B0919E007E
:10173000B0939B00B0939C00B0919A00B093A3002B
:10174000B1E0B093A40018E12CE0B0916D00B117A6
:1017500040F07D7F746020936F00BFEFB0939B00DB
:1017600006C0B0919600B13008F0AFCF60C072FFF4
:1017700011C067FD0FC0B0916F00BA9519F47B7F5F
:101780007860A3CFB0936F00B0919600B13008F0AD
:101790009CCF4DC020927000B091990002E810914A
:1017A000D600112309F003E0B01708F040C085FF10
:1017B00004C0B0916800BB23D1F1B091BA00B3303E
:1017C00081F495FD03C087FD04C00BC087FF01C0F5
:1017D00008C067FD06C06068B0919E00B0939B0092
:1017E00089CF00EF67FF05C0B0919E00B0939B00CA
:1017F00000E2B0917B00B01708F467CF67FF17C015
:101800006F779F7D87FD90627460B2E1B0936F0047
:10181000B0919E00B0939B0058CFB0917000B395EB
:10182000B0937000B0919600BB2309F002C02092E3
:101830007000F89437DC8090B900B2E0B093B90042
:1018400081DC8092B9002092610020926200209297
:101850006300522C2092640020929F0060E070E0B0
:101860007894E8D61FDC0091D600002319F0919AF5
:10187000909A939AB7E0B06CB7B9B6B1B460B0685B
:10188000B6B985FF05C0B0917000B43008F026CD20
:1018900056CEEDE0F0E023D00A3509F01BC0EEE0B3
:1018A000F0E01DD0053A09F015C03AE0A2EBB0E037
:1018B000E3E0F0E014D00D9331963A95D9F739E191
:1018C000AEEBB0E0EFE0F0E00AD00D9331963A9540
:1018D000D9F702C0F4DB0AD0E8E2F0E00895E1991C
:1018E000FECFEEBBFFBBE09A0DB308951ED03AE0E9
:1018F000A2EBB0E0E3E0F0E00D910FD031963A9525
:10190000D9F739E1AEEBB0E0EFE0F0E00D9105D0B2
:1019100031963A95D9F712D00895E199FECF0DBBD3
:10192000EEBBFFBBE29AE19A0895EDE0F0E00FEF25
:10193000F4DFEEE0F0E00FEFF0DF0895EDE0F0E02F
:101940000AE5EBDFEEE0F0E005EAE7DF089530912D
:10195000AE000091AF00313011F40093B600323088
:1019600011F40093B700333011F40093B800343011
:1019700011F40093C400353011F40093B9003630EF
:1019800011F40093D500373011F40093CE003830B5
:1019900011F40093BA00393011F40093BB0008959C
:1019A00025E04AD62A95E9F7089551D653D655D65B
:1019B00057D63CD64CD64ED650D652D637D647D62A
:1019C00049D64BD64DD608954BD647D643D63FD6AB
:1019D0002DD646D642D63ED63AD628D641D63DD684
:1019E00039D635D608958090AE009090AF002FD6AE
:1019F0002ED62DD61BD68A94D1F732D617D69A94E6
:101A0000E1F70895F894D1DF7894CADFC9DFB1E037
:101A1000B093AE00B1E0B093AF002092B000F89464
:101A2000E2DF7894B5E06B2E7090960005D6B09109
:101A300096007B16C9F7B13018F0BF3F40F107C0E0
:101A400086DFF89453DFB1DFB8E0B1BDA9DF6A9457
:101A500059F7B091B000B395B093B000B33008F42B
:101A6000DECF9EDFB091AF00B395B093AF00F89496
:101A7000B091AE00BA95EEE3F0E0EB0FF21D0491E9
:101A800078940395B091AF00B01708F4C6CF88DF03
:101A900087DFB091AE00B395B093AE00B091AE00C9
:101AA000BA3008F4B7CF0BDBF89420DFB8E0B1BD53
:041AB00077DFC9CB48
:00000001FF
